:10000000F52B00308A000408840A82070034523439
:1000100048342034203420343D34203430343034DB
:100020002E343034203425340034543465346D3467
:10003000703420343D342034303430342E34303475
:1000400020344334003420346E346F34203472341E
:100050006534733470342E34663472346F346D34D6
:100060002034443448345434323432340D340A3475
:100070000034523441343234203455344134523413
:10008000543433342034393436343034303420343A
:100090006234643473342034003443346834653457
:1000A00063346B34733475346D34203445347234B6
:1000B00072346F34723421340D340A3400345434C1
:1000C00069346D34653420346F34753474342134BC
:0200D0000034FA
:100140000D3027210A302721080064008001840A2D
:100150000406031900340406A628BF003F088400E3
:1001600083130008031908003F08840000082721B2
:1001700001308312BE003E08BF07AE28831605106B
:100180000510831205104130BD00EE30BC00BC0BE1
:10019000C728BD0BC7280000831205141330BC000C
:1001A000BC0BD028D328831605140800BF00831287
:1001B0003F0884000120003A031908003F0884002A
:1001C0000120272101308312BE003E08BF07C7303F
:1001D000BE00EA28BE0BE928ED28EE28D7281A3001
:1001E0008312BE00BE0BF22800008312051808001F
:1001F0003530BE00BE0BFA288312051C08002130E2
:10020000BE00BE0B012901308312BC000030BD00CE
:100210000800BE003C0884000120003A031922298E
:100220003C0884000120BD003E0884003D08831383
:1002300080000130BD003D08BC070130BD003D0815
:10024000BE070A293E088400831380010800831238
:10025000BD003D09BC003C08A0000830A10005110C
:100260003E21A00C031836290515372905113E211A
:10027000A10B312905153E213E214A291C30A2003F
:100280000000000000000000A20B40290000000058
:1002900000000800000008004408450403197929FB
:1002A000C901C90AC51B602901300310C40DC50D61
:1002B000FF3E031D55290130C8004808C9075229CF
:1002C00045084702031D662944084602031C6E299F
:1002D0004408C6024508031CC703C70201300310C7
:1002E000C50CC40CFF3E031D6F290130C902031D5C
:1002F00060294708C5004608C4000800C101C201C2
:100300003C083D040319B529C301C30ABD1B942948
:1003100001300310BC0DBD0DFF3E031D89290130C6
:10032000C0004008C307862901300310C10DC20D6B
:10033000FF3E031D95293D083F02031DA1293C08EE
:100340003E02031CAA293C08BE023D08031CBF0351
:10035000BF02411401300310BD0CBC0CFF3E031D55
:10036000AB290130C302031D94294208BD00410896
:10037000BC000800BE019901C001BF01831205182D
:10038000CD290130BC003C08BF0765303F02031C8B
:10039000CB299901990ACC29BE291330BC00BC0B8A
:1003A000CF29D22983120518E6290130BC00400864
:1003B000073C013EDD290310BC0DFF3E031DDB2978
:1003C0003C08FF3ABD003D08BE05052A0130BC00CF
:1003D0004008073C013EEE290310BC0DFF3E031D03
:1003E000EC293C08BD003D08BE04BF018312051C7A
:1003F000052A0130BC003C08BF0765303F02031CE2
:10040000032A9901990A042AF6290130BC003C0804
:10041000C00708304002031CBD293E080800013017
:1004200085000130831685008312850183168510AF
:100430008312851083160511831205158316051086
:1004400083120515A001A101A201A301A401A50128
:1004500085100330CC000830CB007730CA00CA0BBF
:100460002F2ACB0B2F2ACC0B2F2A83128514033073
:10047000CC000830CB007730CA00CA0B3D2ACB0B2A
:100480003D2ACC0B3D2A01308312A4070318A50A8C
:100490000030A50700302502063003192402031C92
:1004A000282AA401A5012408263E84008313800184
:1004B0000130A4070318A50A0030A5070030250263
:1004C000153003192402031C532AA0201030831274
:1004D000CC003930CB000D30CA00CA0B6D2ACB0BD3
:1004E0006D2ACC0B6D2A742AA02033308312CA00E7
:1004F0004A08BC00263009212630AD20A020153046
:100500008312CC004B30CB00BE30CA00CA0B862A07
:10051000CB0B862ACC0B862A00008312A401A501EE
:10052000962BBA21CA004A089600BA21CA004A0886
:100530009500BA21CA004A089800BA21CA004A08A0
:100540009700BA21CA004A08940019080319AA2A78
:100550005930952B15081607CA0018084A07CB0012
:1005600017084B071406031D942B0F30CA004A08C6
:10057000BC00263009211608CA00CB014A088C00AD
:100580004B088D001508CA00CB010C08CD00CC012A
:100590004A084C048C004B084D048D001808CA0012
:1005A000CB014A088E004B088F001708CA00CB0108
:1005B0000E08CD00CC014A084C048E004B084D04B7
:1005C0008F0080300F02013003190E02031CF32A42
:1005D0002D30CA004A08AC00FF300E058E007F3077
:1005E0000F058F00F72A2030CA004A08AC000A30F5
:1005F000C4000030C5006430BC000030BD000F08EE
:10060000BF000E08BE007E213D08C7003C08C600A2
:100610004C214408303ECA004A08AD000A30C400EC
:100620000030C5000A30BC000030BD000F08BF001C
:100630000E08BE007E213D08C7003C08C6004C21C4
:100640004408303ECA004A08AE000A30C4000030F8
:10065000C5000F08C7000E08C6004C214408303EF4
:10066000CA004A08B000B030CA004A08B10043309E
:10067000CA004A08B2002030CA004A08B300B401D8
:100680002630AD200130CA004A08BC0026300921BE
:100690000A30C4000030C5006430BC000030BD002A
:1006A0000D08BF000C08BE007E213D08C7003C08B5
:1006B000C6004C214408303ECA004A08AD000A304A
:1006C000C4000030C5000A30BC000030BD000D0879
:1006D000BF000C08BE007E213D08C7003C08C600D4
:1006E0004C214408303ECA004A08AE000A30C4001B
:1006F0000030C5000D08C7000C08C6004C21440896
:10070000303ECA004A08B0002530CA004A08B1008D
:100710000D30CA004A08B2000A30CA004A08B300C5
:10072000B4012630AD20962B4730D6201530CC00B2
:100730004B30CB00BE30CA00CA0B9C2BCB0B9C2B82
:10074000CC0B9C2B000001308312A4070318A50AD0
:100750000030A5070A30C4000030C5006430BC007A
:100760000030BD002508BF002408BE007E213D08E2
:10077000C7003C08C6004C214408303ECA004A0865
:10078000A6000A30C4000030C5000A30BC000030AA
:10079000BD002508BF002408BE007E213D08C7001B
:1007A0003C08C6004C214408303ECA004A08A70055
:1007B0000A30C4000030C5002508C7002408C60060
:1007C0004C214408303ECA004A08A8002030CA0024
:1007D0004A08A900AA012630AD20BE20EF203C081F
:1007E0003D04031D912A1D30952B83132430840072
:1007F0003C30A5200C3084001A30A52083010F2A3C
:02400E00F13F80
:00000001FF
